:020000020000FC
:1000000057CEC2C10000000020C0000094C0000014
:1000100000009EC000000000000000000203040673
:10002000080C10182030406080000406080C1018DE
:100030002030406080A0C00000070F1F3F000D0D62
:100040000403060D0503030202004FB662FD0EC055
:10005000552009F00994C52DC095089483FDC795D6
:10006000C4BDC093A10064604FBE1895C0916400E8
:10007000089483FDC795C4BDC093A1006B7FC09158
:100080006400CF3F09F420C070FF02C082FD05C0AC
:100090004FBE9598AC98C098189575FD0EC065FD3B
:1000A0000CC0C091B300C0FD9498C1FDAD98C2FDD5
:1000B000AB98CAEFC095CA95F1F79598AC98C098DF
:1000C0002092A1004FBE189524BCCC27C064C8BFA5
:1000D0006460F6CFC0CF70FFBECF65FDBCCF959AF0
:1000E000BACF70FFB8CF65FDB6CFAC9AB4CF70FF72
:1000F000B2CF65FDB0CFC09AAECF949A70FFABCFB0
:1001000065FDA9CFC7E0CA95F1F7959AA4CFAD9A3E
:1001100070FFA1CF65FD9FCFC7E0CA95F1F7AC9AFC
:100120009ACFAB9A70FF97CF65FD95CFC7E0CA9580
:10013000F1F7C09A90CF4FB6C9B7CF7EC9BF6E7FD7
:10014000CCB5CE0DDDB5DF1DDBBDCABD4FBE1895EC
:100150003FB68F7EABB7A074A2118061A0E0ABBFA9
:10016000A9B7AE7FA9BF7894A0916800AA2341F0F7
:1001700085FD2AC0A0916800AA95A093680024C0BC
:1001800040E050E085FD14C0A0B396FDA095A2FD0F
:100190004FEFA3E096FDA2E0A5BFAA27A064AABFE7
:1001A0008D7FA0B396FDA095A2FD5FEF451741F7A7
:1001B000A0E461FDA093680085FD03C0A0E4A093C6
:1001C000680040939700816085FD0EC0A091690092
:1001D000AA2331F0A0916900AA95A093690004C0F8
:1001E0008061AA27A064AABF80FF0AC0A0919700DF
:1001F0004A2F61FF8E7F85FD01C000C040936100E2
:100200004091B600443009F004C0A0916100A09371
:100210006300A52DA03408F06860A0916000A3954C
:10022000A093600051F0F894A9B7A160A9BF84FF22
:1002300002C0A0E4ABBF3FBE1895A0917400A39587
:10024000A093740042E050916800552329F085FF87
:1002500003C05A9550936800A0919700A13018F000
:1002600020929A000DC020929B002092A500A091A0
:100270009A00AF5FA0939A0018F0AFEFA0939A0096
:10028000B09061005091B600523049F466FF91F091
:10029000A2E3BA1678F0A0918700A09361005330D2
:1002A00049F466FF39F0A2E3BA1620F0A091C2002B
:1002B000A0936100509162005B1521F010F05A95F7
:1002C00001C05395509362004A95D1F65091A50014
:1002D000539509F45A955093A500A091A600AA95AC
:1002E000A093A60009F046C0A1E0A093A60045E0B7
:1002F000A091A7005A17F0F1A091A8005A1728F46E
:1003000041E0A3E0A093A60007C0A091A9005A175E
:1003100018F441E04093A600D0909D00C090630087
:10032000DC14A8F0A091B600A430D9F066FD0FC08F
:10033000C0929D00539511F0A091A700A093A50035
:10034000A1E0A093A600ACE3A093620013C0A0912B
:100350009D00A40F20F45FEF50939D0002C0A09376
:100360009D00A0919D00AF3F29F4AFEFA0939B00AB
:10037000A093A500F894A9B7A160A9BF84FF02C00B
:10038000A0E4ABBF3FBE18953FB64CB55DB58F7EC0
:10039000ABB7A074A2118061A0E0ABBFA9B7AE7FDC
:1003A000A9BF789481FD23C0A2E096FDA3E0A5BF7C
:1003B0008260A0B396FDA095A2FF05C040936500A2
:1003C000509366001CC1A3E096FDA2E0A5BFAA273A
:1003D000A064AABF8D7F85FF01C004C140E0A0B327
:1003E00096FDA095A2FDFEC040939700EDC0A3E04E
:1003F00096FDA2E0A5BF8D7F61FF71C0A2E096FDD2
:10040000A3E0A5BFAA27A064AABF82604093920080
:1004100050939300A09090004A19B09091005B090E
:10042000BB24A22C4C38520518F42092960049C0E7
:10043000A091D600AA2359F1483C520528F4A0E126
:10044000BA2EAAE0AA2E23C04836A1E05A0728F403
:10045000A8E0BA2EAFE0AA2E1AC0403DA2E05A078B
:1004600028F4A4E0BA2EAEE1AA2E11C0403AA5E0CD
:100470005A0728F4A2E0BA2EACE3AA2E08C04839E5
:10048000A8E05A0720F4A1E0BA2EA8E7AA2EC42EAD
:10049000A0919400CA1AD52EA0919500DA0ADD2009
:1004A0002AF4AFEFC094D094CA1ADA0A20929600C8
:1004B000A8E0A210A0E0CA14DA0618F4A1E0A09304
:1004C0009600409394005093950040919200509173
:1004D0009300409390005093910002E075C0A0916A
:1004E00065004A1BA09166005A0B94FD60C093FD05
:1004F0005EC092FD5AC086FF03C0D52EC42E0CC02C
:100500005695479591FD51C05695479590FD4DC024
:10051000D52EC42ED694C79461FD19C0AC2DAC5114
:10052000AD2DA24008F005C0DD2089F4AC2DA85CFB
:1005300070F4A0916700A395AA2311F0A09367001F
:10054000AA3008F44FC02092970081604BC0A09160
:100550006700AA2319F0AA95A0936700A22C5091D6
:10056000BC0097FD02C0A090CA00AAEFAA0EA22D5F
:10057000A21DCA18DA0A4FB74170442319F040E0AF
:1005800050E015C0AFEFCA16D20418F04FEF50E09C
:100590000EC0A091AE00CA9E412D000C441F50E039
:1005A00008F012C04FEF50E00FC05695479594FFEA
:1005B00007C0552309F04FEFA42FA6954A0F521DEF
:1005C0004F3F520508F04FEF40939700816061FF65
:1005D00009C0AFE1A095A923AB299A2F8F7DBB203D
:1005E00009F48062A0E4A093680085FF03C0AAE03C
:1005F000A093680061FD03C085FD01C08F7E85FD6D
:1006000003C0A0E2A0936900F894A9B7A160A9BFB4
:1006100084FF02C0A0E4ABBF3FBE189511E00AC042
:1006200013E008C01AE006C01EE104C014E602C0D0
:1006300018EC00C005E1BB27BA95F1F70A95D9F788
:100640001A95C1F708952AE338E709C020E33CE88A
:1006500006C02AE234EB03C025E238EC00C012E009
:1006600095FD9F7D95FF9062BB27AD9ABA95F1F7F6
:10067000AC9ABA95F1F7AC98BA95F1F7AD98BA95EE
:10068000F1F7959AB091AF00BA95F1F79598B7E860
:10069000BA95F1F71A9521F7022FB22FBA95F1F713
:1006A0000A95D9F73A95D9F6AD9A0895221B39E003
:1006B000001F3A9509F40895221F211B18F4210FF9
:1006C0008894F6CF0894F4CF622C722CB0E0889412
:1006D000B395221F331FE0F7379527958894912E05
:1006E000802E020B130B10F4192D082D10F4889492
:1006F00001C00894661C771CBA9571F7172D062D5A
:100700000895322D11232AF43A9500951095031B74
:10071000130BF894029F712C002D129F912C802CAA
:100720007894780C172D921C292DB4E06B2E269509
:10073000179507956A94D9F7332321F00095109502
:10074000031B130B08950091B600043009F474C024
:10075000B0919700B95198F0B72FB67081F466FD4B
:100760002BC005E09090C800B92DBA9521F00AE0A1
:10077000BA9509F002E1B0917B00B01BE0F066FF92
:100780000AC0B0919F00B0939D00BFEFB093A50049
:10079000B1E0B093A600B0916100B09363002092E5
:1007A0007F0020928000209281002092820020927F
:1007B00083006F7B41C060649090C800B92DBA95EA
:1007C00079F4B0916200B095BB1FBB1F1B2FB7958A
:1007D0000B2FB12FB170B3951B2FB02FBE7F25C04B
:1007E000B92DBA95BA9581F4B0916200B095BB1F4E
:1007F000BB1FBB1F1B2FB7950B2FB12FB370B3952A
:100800001B2FB02FBC7F14C0B0916200B095BB1FEE
:10081000BB1FBB1FBB1F1B2FB7950B2FB12FB77073
:10082000B395B3951B2FB02FB87FB0540B2F12097F
:1008300000937F0010938000089510917B0016951F
:1008400000917A000795B0917F00B01B0B2FB091FB
:100850008000B10B1B2F28F40038BFEF1B0740F0BE
:1008600009C00F37120508F405C00FE710E002C0F9
:1008700000E81FEF00938400109385000895009115
:100880008400B09181000B0F10918500B09182001F
:100890001B1F20E03091850033230AF42A95B09184
:1008A00083002B1F1AF4203F40F00AC02F3008F4B9
:1008B00007C00FEF1FEF2FE003C000E010E020EFB4
:1008C00030916300B0919C003B1718F4323030F047
:1008D00009C0B0918500BB235AF004C0B0918500D7
:1008E000BB2332F400938100109382002093830095
:1008F00008952091D80000918400000F1091850088
:10090000111FFFDE11232AF40038BFEF1B0740F050
:1009100009C00F37120508F405C00FE710E002C048
:1009200000E81FEF002352F0B0916200B01B0B2FC4
:1009300018F0013008F00AC001E008C000950F5F10
:10094000B09162000B0F08F001C00FEF009386001A
:1009500008952091D9000091820010918300D1DE8A
:1009600011232AF40130BFEF1B0740F009C00F3FED
:10097000120508F405C00FEF10E002C001E01FEF00
:10098000112352F0B0918600B01B0B2F18F00130EC
:1009900008F00AC001E008C000950F5FB091860022
:1009A0000B0F08F001C00FEF0093630008950FEFE5
:1009B000677F71FD29C072FD09C06860B0917B003E
:1009C000BA3020F0B52DB03408F4677FB091D5006F
:1009D000BB23D1F0B0917B00BB23B1F00FEF10919E
:1009E0007B0064DEF894B091730072FDB5E00B9F5C
:1009F000112D002D7894112309F00FEFB0919F0075
:100A00000B1710F400919F0000939E000895009131
:100A10007A0010917B0000541140B0919E0010F4B8
:100A2000BA9501C0B39511F0B0939E000895EFD32D
:100A3000B2E073FDB1E0B7B9B6B1B068B064B6B9B1
:100A4000EDDDB2E073FDB1E0B7B9B6B1B068B06446
:100A5000B6B9B6B1B6FDFDCF04B115B1B6B1BF7729
:100A6000B6B926D424E72093AA00222309F441C072
:100A700030E03093AB00732E7694622E6694620E53
:100A8000731E262D372D0217130778F08090AA00C9
:100A9000B4E7B80DB093AA008090AB00B0E0B81DE9
:100AA000B093AB00260D371DEECF8090AA0090903A
:100AB000AB001091AB0016950091AA000795169512
:100AC000079523E0169507952A95E1F72091B70041
:100AD0002A9529F42092AA002092AB000AC02A95F8
:100AE00021F0800E911E2A95E1F78092AA00909243
:100AF000AB0008952091B700B6B1B6FDFBCF04B1AD
:100B000015B1B6B1BF77B6B9B091AC00B395B0939B
:100B1000AC00B83060F12092AC00B091D400BB239F
:100B200021F1112329F0B091AD00BF3F61F009C060
:100B3000B091AD000B1739F020F4BB2321F0BA952A
:100B400002C0B395E1F300919C00B093AD00B838BA
:100B500050F400ECBD3738F400E8B23720F400E47C
:100B6000B73608F400E000939C00777F08952130A9
:100B7000B1F00F3FB3E01B0790F4B4E7BB2379F06B
:100B8000B091AA000B17B091AB001B0740F4B091D5
:100B90009C00BB2359F0BA95B0939C0007C0B0915C
:100BA0009C00BF3F19F0B395B0939C0000919C004E
:100BB000B0916300B01B10F400916300B0919D00F0
:100BC0000B1750F000919D00B0919D00BF3F21F0A8
:100BD000B0919D00B0939C00502E00936400B091A2
:100BE000AC00B73009F47860089502E3F894B0914E
:100BF000DA000B9F012D000C001F7894B0919C002F
:100C00000B1710F000919C000093610000936300AB
:100C1000502E0093640000939F00089520927A0064
:100C2000B0EFB0937B000895F8940CB51DB52091FA
:100C30007400789430917500609076000093750090
:100C400010937600031B160971FD03C076FD81C069
:100C50002BC070907700209377002709222311F092
:100C60000FEF1FEF8090780090907900309378001C
:100C7000609279006918161910937C000091750034
:100C8000109176000819190920917A0030917B00A3
:100C900036952795020F131F10F40FEF1FEF0093E7
:100CA0007A0010937B0029C020917A0030917B005C
:100CB0003901B4E08B2EB2E09B2E343010F08A94D0
:100CC0009A94383010F08A949A94769467948A941F
:100CD000E1F726193709992021F0169507959A947E
:100CE000E1F7200F311F20937A0030937B0028F426
:100CF0003FEF30937A0030937B00323008F4706419
:100D000071FF02C0B3E00DC0B091C6000091710048
:100D1000023838F0B395003A08F0B395B63008F0D1
:100D2000B5E09B2EB4E08B2E10917B0000917A00F1
:100D300024E0169507952A95E1F70819120928F07D
:100D4000B02FB250B12FB20910F402E010E09801B8
:100D500026C020917A0030917B0039017694679407
:100D60006694669466942619320906950695200FB6
:100D7000321D20937A0030937B00323008F07F7B65
:100D800004E0369527953695279526952695201BC0
:100D900010F0223008F422E089019090C60060FD36
:100DA000FECFE0908C00F0908D006160B9B7B0612B
:100DB000B9BF380176FD44C07694679400938C00E7
:100DC00010938D00B92DB330E1F0B0FD04C0060DD5
:100DD000171D930106C0000F111F0250120922E0D7
:100DE00030E0B92DB33068F020938E0030938F003F
:100DF000009388001093890060928A0070928B00A3
:100E00003DC000938E0010938F0020938800309394
:100E1000890060928A0070928B0071FF10C0B091BF
:100E20006D00B33060F000918F0010917C0015953B
:100E3000010F28F022F020928E0000938F001EC038
:100E4000669400938C00B92DB33091F0B0FD03C0CF
:100E5000060D262D03C0000F025022E0B92DB3303D
:100E600038F020938E000093880060928A0006C0BC
:100E700000938E002093880060928A0000917D008C
:100E800002FD0350013029F495FD0AC0B6E0B7B960
:100E900009C0023019F4B7E0B7B904C095FDF6CF28
:100EA000B0E0B7B90091A400000F10F4BBE60B2727
:100EB0000093A40060FDFECFB2E0B0936E006160CD
:100EC000B9B7B061B9BFB72FB670A1F020917A0061
:100ED00030917B0036952795F8940CB51DB5020F1F
:100EE000131F1BBD0ABD6160B0E1B8BFB9B7B061E7
:100EF000B9BF78940895606120927E0020E067FD7C
:100F000020E206C0606120927E0020E267FD20E0C2
:100F1000789401E076FD11C0B72FB67009F06F7EAE
:100F2000B0917B00B55048F002E0B55020F003E0EE
:100F3000B55008F006E071FD0AE060FD12C0B09106
:100F40007E00BB2371F071FF08C0B0916D00B3301B
:100F500020F0B0916E00BA9519F4789470615CC07D
:100F6000AEDF789400000000F89476FD16C0109172
:100F70007B00173008F017E0B5E01B0F72FD10E1A1
:100F800083FF110F62FF110F71FD12E8B4B560907D
:100F9000A100B61990F2B10B80F2B0B7B77FB0BF25
:100FA000B8B1B0B7B860B0BFB0917E00B395B093A0
:100FB0007E00B8B176FD06C0B1E071FDB2E0BA9531
:100FC000F1F7B8B1B072B21709F01BC071FF05C0DC
:100FD00003950A3008F00395B0CF64FF99CF6F7E78
:100FE0003CB56DB470907A0080907B00370D681C22
:100FF0006BBC3ABD6160B0E1B8BFB9B7B061B9BF11
:1010000087CFB0916D00B23008F482CF64FD80CFFD
:101010000A9509F092CF7F7E20918E0030918F004B
:10102000F894B0E1B8BF0CB51DB5020F131F1BBD7E
:101030000ABDE0908800F09089006160B9B7B061A6
:10104000B9BF7894B72FB67039F0B0916D0072FFC8
:10105000B395B0936D0009C074FF07C067FD05C06C
:1010600064FD03C0BF91BF91D6C4089500E063FF43
:1010700003C064FF01C001E0F89410917100B7E073
:101080001B9F212D102D7894200F269517952695BE
:1010900017952695179510937100183718F4B8E72F
:1010A000B093710000917100B09172000B1720F0A5
:1010B00060629598AC98C09860FDFECFE0908A0081
:1010C000F0908B006160B9B7B061B9BF0895B2E02C
:1010D00095FD07C0F894B0937D00AD9A94987894EC
:1010E000E5C0F894B0937D00AD9AAB987894DEC0DB
:1010F000B3E082FF24C095FD11C002E0F894B093E4
:101100007D00E7E8F0E00093B300C098AB9A62FF7F
:1011100002C0AC9A01C0AD987894C8C002E0F894BF
:10112000B0937D00E7E8F0E00093B3009598949ABF
:1011300062FF02C0AC9A01C0AD987894B7C095FD2B
:101140000BC0F894B0937D00E1E7F0E0C09862FF37
:1011500001C0AC9A7894AAC0F894B0937D00E1E7FE
:10116000F0E0959862FF01C0AC9A78949FC0B4E01B
:1011700095FD07C0F894B0937D00949AAB9878944D
:1011800095C0F894B0937D00AB9A949878948EC0F3
:10119000B5E082FF24C095FD11C001E0F894B09342
:1011A0007D00EDE7F0E00093B300AC98AD9A62FFEC
:1011B00002C0959A01C09498789478C004E0F8949D
:1011C000B0937D00E1E9F0E00093B300AC98AD9AF4
:1011D00062FF02C0C09A01C0AB98789467C095FDC9
:1011E0000BC0F894B0937D00EBE6F0E0AC9862FFA2
:1011F00001C0959A78945AC0F894B0937D00E7E7BF
:10120000F0E0AC9862FF01C0C09A78944FC0B6E09D
:1012100095FD07C0F894B0937D00AB9AAD98789493
:1012200045C0F894B0937D00949AAD9878943EC0F0
:10123000B1E082FF24C095FD11C004E0F894B093A2
:101240007D00E1E9F0E00093B3009598949A62FF85
:1012500002C0C09A01C0AB98789428C001E0F8940D
:10126000B0937D00EDE7F0E00093B300C098AB9A37
:1012700062FF02C0959A01C09498789417C095FDBA
:101280000BC0F894B0937D00E7E7F0E0959862FF1B
:1012900001C0C09A78940AC0F894B0937D00EBE640
:1012A000F0E0C09862FF01C0959A78946F7D089530
:1012B0002AE630E0F9012092B3009598AC98C098E6
:1012C000949AAD9AAB9A6B7F0895A4EBB0E007E0D7
:1012D0000D9307E00D9301E00D9304E00D930FEFE4
:1012E0000D930D930BE00D9302E00D9301E00D9330
:1012F00001E00D93A0ECB0E001E00D9300E00D9350
:1013000004EB0D930FEF0D930D930D9303E00D93ED
:101310000FEF0D9301E00D930FEF0D9305E20D9389
:1013200000ED0D9308E70D9308EC0D9304E00D9389
:101330000FEF0D9301E00D9300E00D930AE70D937D
:1013400007E00D9300E00D9301E00D9300E00D9395
:101350000FEF0D9308952091BB008B7F233009F48C
:101360008460B091BC009F7DB1FD90629F7BB09185
:10137000BD00B1FD9064223011F0886001C0877F0C
:1013800008950A95E00FF21DB4910895ECE1F0E0A4
:101390000091B400F6DFB093D800ECE1F0E00091EA
:1013A000B500EFDFB093D900EAE2F0E00091BA00B7
:1013B000E8DFB093DA000091D300002309F403952D
:1013C000013108F001E1B02FB00FB00FB093A700CA
:1013D0001B2FB10FB10FB00FB093A800B10FB00F1A
:1013E000B00FB093A900B091D0000FEF1CE0B23065
:1013F00011F400EA1AE0B33011F402E815E00093AA
:10140000720010937300E8E3F0E00091D700B9DFB9
:10141000B093A200089508952091CA003091CB00A6
:10142000B091BC00B33009F43E5097FF02C020E0F9
:101430003FEFB32FB21B6B2EB25810F4B2E86B2EF5
:1014400000E00395609EB12DBD57D8F30093AE0028
:1014500008959068E1DFE8D820E030E0B0E16B2E3D
:10146000DFD8B09197002B0F321D6A94C9F7B4E012
:1014700036952795BA95E1F7822E9F77CDDF0895AF
:10148000F894E3E0F0E0B9E0B7BFB491B078C1F30D
:10149000F894A895B1B5B861B1BDB0E0B1BDB4E004
:1014A000BEBFBFE5BDBF04DFB0E0B8BBB1E1B7BBB5
:1014B000B8E2B5BBB8E3B4BBB0E1B2BBB0E3B1BB1B
:1014C0002224A0E0B0E02D92AA31E9F7A0E6B0E036
:1014D0000FEF2D920A95E9F7B1E0B093A400F5DE85
:1014E000CFD2B6B1B460B6B90091CC000093AF00D2
:1014F000B1E0B0936A00F8949BD8A5D895D8A6D847
:1015000093D8A7D891D84BD393D892D88FD8F894A2
:101510000AEF1AEFA0B396FDA095A2FF1FC01A957F
:10152000C9F70A95B1F7E0E0FCE1B591B43E39F4B2
:10153000B591B03E21F4B591BF3F09F40CC0E0E095
:10154000F395F395B591B83F49F4B591B43931F4B9
:10155000B591BA3A19F4EE27F6950994FCDE16DF38
:101560005ADF5ADF0091CC000093AF00A1DEB2E059
:10157000B3BFB2E0BEBDB2E0B5BDB1E5B8BFB9BF63
:10158000B0B7B77FB0BFB8B1B0B7B860B0BF46D8DA
:1015900078944DDAB3E096FDB2E0B5BFB0E4BBBFDE
:1015A000BB27B064BABF8D7F43D8626033E02CE0C4
:1015B000B0919600BB2321F42CE03A9509F4A7CF13
:1015C00033D880FFA4CF8E7FB0919700B23078F3EC
:1015D000B92FBF710091990000939800B0939900C2
:1015E000B01729F72A9521F76D7FB3E096FDB2E099
:1015F000B5BFBB27B064BABF8D7FB091D600BB2307
:1016000021F48062B92FB0709B2F8F7B20926700EE
:101610000DD885FF05C0B0916700BA3008F080642E
:10162000FFD702E085FF01C000E0B0919700B0173E
:10163000B8F3F89408D807D806D87894F9D7209248
:101640008700EED7B091C000B13008F46EC0B09101
:101650006A00B13008F469C085FD18C0B0919700E8
:10166000BF3F08F462C0F894F7D77894DFD7B09101
:101670009700B130C0F7F894E6D7D4D7E4D7789480
:10168000D5D7B0919700BF3FB0F3BBC2B8E09B2E57
:101690009068F894C1DE7894C9D7F8949F77BCDE3F
:1016A00080909700B0919700BF37789408F445C0B8
:1016B000B5D7F894D1D778949A9451F7CADEB82D5B
:1016C000B550B093CB00B4D7F89407D26DD27894CC
:1016D000BAE09B2E9068F8949FDE7894A7D7F89490
:1016E0009F779ADE80909700B0919700BF377894EB
:1016F00078F794D7F894A7D795D7A5D778949A94E4
:1017000049F7A7DEB82DBB5FB093CA0091D7F89414
:10171000E4D159D278948AD7F8947EDE7894B09147
:101720009700BF3F08F498CF6CC200919700B0912A
:1017300087000B1710F00093870078D701E0B09175
:10174000BC00B35009F405E0B0919700B01708F061
:1017500078CFF89481D780D77FD7789469D72092B3
:101760006A0020926B0020926C00B0916B00B395E0
:10177000B0936B00BF3F69F5B0916C00B395B09327
:101780006C00B091CE0009E1BA9559F002E3BA9528
:1017900041F00DE7BA9529F00AEFBA9511F02092C1
:1017A0006C00B0916C00B017A0F0B0916C00BA95CD
:1017B000B0936C00B4EBB0936B00B091CD00B093DC
:1017C000AF00F89449D77894B091CC00B093AF00B3
:1017D0002DD728D7B0916800BB2319F485FF01C02D
:1017E00096CE01E085FD01C006E0B0919700B017EC
:1017F00008F4BBCF1BD7B0916800BB2309F487CE98
:10180000F89456DD209261002092620020926300DD
:10181000522C209264002092A3007894B091B900D9
:10182000BB0FB093A00020927F00209280002092F6
:10183000810020928200209283002092AC0060E020
:1018400070E020927100B8E0B093AC007860E6D60A
:10185000B2E073FDB1E0B7B9B6B1B068B064B6B983
:10186000B6B1B6FDFDCF04B115B1B6B1BF77B6B90B
:10187000112309F00FEF0093AD003CD9B8E0B0930D
:10188000AC0078608090BB00B2E0B093BB0063DD39
:101890008092BB00F894BFEFB0939C00A6D9B091A2
:1018A0006100B0939C00B0939D00B0939E0078942B
:1018B000B1E0B0936100B09363005B2EB09364001D
:1018C000B093A600B0919B00B093A500B091BC006E
:1018D000B33019F49F7D87FD906271607260209231
:1018E0006D0095DCA5DC9AD99FD998D99DD996D958
:1018F00006C0F89430DD78942092AC00777F02DB4C
:1019000022D7B4DBE4DB90D9F6DA66FD96D776FF12
:101910004ED876FD7CD8AADBEBDB86D9F3DA66FD00
:10192000AED7A4DB24DC80D9E6DA66FDE2D79EDB05
:101930002FDC7AD9E7DA66FD0CD898DB68DC74D93D
:10194000DADAB2E073FDB1E0B7B9B6B1B068B0644D
:10195000B6B98CDB6DDC68D9CDD871FF20C067FDCE
:101960001EC0B0919F00B0939C00B0939D00B091B9
:101970009B00B093A500B1E0B093A60018E12CE065
:10198000B0916D00B11728F07D7F746020936F00D7
:1019900006C0B0919700B13008F0B1CF46C072FFD9
:1019A00010C067FD0EC0B0916F00BA9511F47B7F37
:1019B000A0CFB0936F00B0919700B13008F09FCFE7
:1019C00034C020927000B0919A00B13058F0B091BC
:1019D0009F00B0939D00B0919B00B093A500B1E033
:1019E000B093A600B0919A000AEFB01708F01DC09E
:1019F00085FF04C0B0916800BB23B9F000EF67FF1A
:101A000005C0B0919F00B0939C0000E2B0917B00B4
:101A1000B01708F474CFB0917000B395B093700014
:101A2000B0919700BB2309F002C020927000F89497
:101A30003FDC8090BB00B2E0B093BB008CDC8092B6
:101A4000BB00209261002092620020926300522C21
:101A5000209264002092A0007E7F7894DFD528DC5D
:101A6000B6B1B460B6B985FF05C0B0916800BB23BC
:101A700009F44DCDB091C100B13008F0D1CD71CE97
:101A8000EDE0F0E023D0053A09F01BC0EEE0F0E015
:101A90001DD00A3509F015C03AE0A4EBB0E0E3E050
:101AA000F0E014D00D9331963A95D9F738E1A0ECD7
:101AB000B0E0EFE0F0E00AD00D9331963A95D9F717
:101AC00002C003DC0AD0E7E2F0E00895E199FECF1E
:101AD000EEBBFFBBE09A0DB308951ED03AE0A4EB35
:101AE000B0E0E3E0F0E00D910FD031963A95D9F7F0
:101AF00038E1A0ECB0E0EFE0F0E00D9105D03196D8
:101B00003A95D9F712D00895E199FECF0DBBEEBBFF
:101B1000FFBBE29AE19A0895EDE0F0E00FEFF4DF09
:101B2000EEE0F0E00FEFF0DF0895EDE0F0E005EA21
:101B3000EBDFEEE0F0E00AE5E7DF08953091B0007A
:101B40000091B100313011F40093B400323011F43F
:101B50000093B500333011F40093B600343011F423
:101B60000093C800353011F40093B700363011F4FB
:101B70000093BA00373011F40093C600383011F4E6
:101B80000093BB00393011F40093D0003A3011F4C7
:101B90000093BC003B3011F40093BD00089525E094
:101BA00047D52A95E9F708954ED550D552D554D545
:101BB00039D549D54BD54DD54FD534D544D546D556
:101BC00048D54AD5089548D544D540D53CD52AD5E1
:101BD00043D53FD53BD537D525D53ED53AD536D596
:101BE00032D508958090B0009090B1002CD52BD5BF
:101BF0002AD518D58A94D1F72FD514D59A94E1F720
:101C00000895F894D1DF7894CADFC9DFB1E0B093CA
:101C1000B000B1E0B093B1002092B200F894E2DFDE
:101C20007894B5E06B2E7090970002D5B091970034
:101C30007B16C9F7B13018F0BF3F40F107C07EDF17
:101C4000F8944BDFB1DFB8E0B1BDA9DF6A9459F772
:101C5000B091B200B395B093B200B33008F4DECFC8
:101C60009EDFB091B100B395B093B100F894B091FC
:101C7000B000BA95EEE3F0E0EB0FF21D049178941A
:101C80000395B091B100B01708F4C6CF88DF87DFA5
:101C9000B091B000B395B093B000B091B000BC303B
:101CA00008F4B7CF12DBF89418DFB8E0B1BD77DFE6
:021CB000E7CB80
:00000001FF
